:020000040000FA
:20000000BC3280BB040008000A8039817F0F02000040000037833A833D8340834383438113
:20002000FF0F040000800000468349834C834F83528393FE28BD28C8401028C80200C803B0
:2000400000E000E114B1EA0880EB09805272110B73FA0371FA025CB86C2880FA0180FA00DA
:2000600080288080808080808080E000E102B1EA0480EB05805272110B736CB8D211DA0151
:20008000E001E114B1EA0880EB09805272110B73FA0371FA025CB86C2880FA0180FA008019
:2000A000288080808080808080E001E102B1EA0480EB05805272110B736CB8D211DA012868
:2000C000C84110E0FFC84210C84310E000C84110E0FFBD28C80100E90100C9000001E002D7
:2000E000299002E100C90100E80000E102B1EA0480EB05805272110B73FA0171FA005CB873
:200100006CE80000E114B1EA0880EB09805272110B73FA04C80010FA05C80110FA06C80234
:2001200010FA07C80310FA08C82010E0FAC840108F8E8D8C8B8A8988BABF0090A9BF0B907F
:2001400093FAA8BF00A0A9BF0BA093FAA828BD28C84010E0FFC80200E80000C80300E00062
:20016000E114B1EA0880EB09805272110B73FA08C82010E001E114B1EA0880EB0980527275
:20018000110B73FA08C82010BBBC88818081828384858687E80000E102B1EA0480EB0580E0
:2001A0005272110B736CB8D211DA01E90100C9000001E002299002E100C90100E80000E145
:2001C00002B1EA0480EB05805272110B73FA0171FA005CB86CE80000E114B1EA0880EB0961
:2001E000805272110B73FA04C80010FA05C80110FA06C80210FA07C80310FA08C82010E0EE
:20020000FAC840108F8E8D8C8B8A8988BA808182832873E842107260980613E101197312D8
:2002200061980613E10219731262980613E10419731263980613E10819731264980613E104
:200240001019731265980613E12019731266980613E14019731267980613E180197312CB83
:200260004210CB43108B8A8988BA8081828384858687E80000E114B1EA0880EB09805272DA
:20028000110B73FA0B80FA0A80B98F8E8D8C8B8A8988BA8081828384858687E80000E114FE
:2002A000B1EA0880EB09805272110B73FA0D80FA0C80B98F8E8D8C8B8A8988BA8081828372
:2002C00084858687E80000E114B1EA0880EB09805272110B73FA0F80FA0E80B98F8E8D8C41
:2002E0008B8A8988BA8081828384858687E80000E114B1EA0880EB09805272110B73FA1130
:2003000080FA1080B98F8E8D8C8B8A8988BA8081828384858687E80000E114B1EA0880EBFD
:2003200009805272110B73FA1380FA1280B98F8E8D8C8B8A8988BABC8A82BCB382BCDC8226
:20034000BC0583BC2E83BC8A82BCB382BCDC82BC0583BC2E83000000000000000000000068
:2003600000000000000000000000000000000000000000000000000000000000000000007D
:2003800000000000000000000000000000000000000000000000000000000000000000005D
:2003A00000000000000000000000000000000000000000000000000000000000000000003D
:2003C00000000000000000000000000000000000000000000000000000000000000000001D
:20100000E054C88000E030C88100B9B9000000000000000000000000000000000000000089
:201020000000000000000000000000000000000000000000000000000000000000000000B0
:20104000000000000000000000000000000000000000000000000000000000000000000090
:20106000000000000000000000000000000000000000000000000000000000000000000070
:20108000000000000000000000000000000000000000000000000000000000000000000050
:20200000E054C80001E031C80101B9B9000000000000000000000000000000000000000076
:202020000000000000000000000000000000000000000000000000000000000000000000A0
:20204000000000000000000000000000000000000000000000000000000000000000000080
:20206000000000000000000000000000000000000000000000000000000000000000000060
:20208000000000000000000000000000000000000000000000000000000000000000000040
:207FE000000000000000000000000000000000004D818C810D826A829382BC82E5820E83E0
:00000001FF
